:020000040000FA
:1000000008288207000080293C2A4129902AE42AF6
:100010008B0109235C235908AA005A08AB005B082E
:10002000AC005C08AD0052275508AA005608AB008A
:100030005708AC005808AD004027851400000000A8
:1000400000000000851085120430870021218516EC
:100050000000000085120030870021218516000075
:100060000000851205185D289323932305185D2849
:100070002D21FF30F800F9000930FA000518592841
:10008000F80B3E28FF30F800F90B3E28FF30F9004E
:10009000FA0B3E28FF30F800F9000930FA00F51895
:1000A0005428F1210330C200F514051C55282D21D8
:1000B0005D2893239323051C3E288A254A08E900DE
:1000C0004908EA004808EB004708EC004608ED0044
:1000D0004508EE004408EF004308F0004924650895
:1000E000DD006608DE006708DF006808E0005208EF
:1000F000E9005108EA005008EB004F08EC004E08F8
:10010000ED004D08EE004C08EF004B08F0004924CC
:100110006608E1006708E2006808E300E401F51BF7
:10012000A32886015D08F1005E08F2005F08F30075
:100130006008F40075100921051500000511013053
:10014000F600F7003228751CFC28F70B32285308FC
:10015000013A031DAE280130F700BE285308023AC9
:10016000031DB5280330F700BE285308033A031DCA
:10017000BC280830F700BE280F30F700760987004A
:10018000870A000005150000051109217108A0006B
:100190007208A1007308A2007408A3006108A400FB
:1001A0006208A5006308A6006408A700A023200831
:1001B000F1002108F2002208F3002308F400F60BF6
:1001C0003228FF30F6002230F100F201F301F40191
:1001D000092176098700870A00000515000005112E
:1001E0005D08F1005E08F2005F08F3006008F400AB
:1001F000051600000512322875145D08F1005E082E
:10020000F2005F08F3006008F40005160000051214
:10021000A52885120030870021217408870021213C
:100220007308870021217208870021217108870047
:10023000212100000000851600000000000085124A
:10024000080000000000000085150000000000000C
:1002500085110000000000000800F5183B29751DFD
:1002600035290D2275110330C200C20B3929023025
:10027000C20042080128C20B3F290530C2004208D3
:1002800001285330B0007030B1006530B200B300C7
:100290006430B4003D30B5002030B600B700B8007F
:1002A000BD006D30BE007330BF005308013A031D1E
:1002B00061292030B9003130BA003030BB00BC00B9
:1002C000072B5308023A031D6D292030B900323044
:1002D000BA003030BB00BC00072B5308033A031DA3
:1002E00079292030B9003530BA003030BB00BC006D
:1002F000072B3130B9003030BA00BB00BC00072BEF
:100300005330B0007430B1006530B2007030B300CB
:100310003D30B4002030B500B600B700B800BC00D6
:100320004830BE007A30BF005408013A031D9F29AF
:100330002030B900BA00BD003130BB00072B540893
:10034000023A031DAB292030B900BD003130BA009C
:100350003030BB00072B5408033A031DB729313056
:10036000B9003030BA00BB002030BD00072B540864
:10037000043A031DC3292030B900BA003130BB0054
:100380006B30BD00072B5408053A031DD0292030DF
:10039000B9003130BA003030BB006B30BD00072BE4
:1003A0005408063A031DDC293130B9003030BA0058
:1003B000BB006B30BD00072B5408073A031DE8292A
:1003C0002030B900BA003130BB004D30BD00072BE2
:1003D0002030B9003130BA003030BB004D30BD00A4
:1003E000072B2030B000B100B700BC00BF00533075
:1003F000B2005730B3004530B400B500B9005030FA
:10040000B6004D30B8004E30BA00BE005530BB00CB
:100410004F30BD0007232A2208002030B000B10071
:10042000B700BC005330B2005730B3004530B400C1
:10043000B500B9005030B6004D30B8004E30BA00AB
:100440005530BB004F30BD004630BE00BF00072313
:100450002A220800FF30F800F9003230FA00F80BC9
:100460002F2AFF30F800F90B2F2AFF30F900FA0B82
:100470002F2A0930FA0008004630B0003D30B100A4
:100480002030B200BD002E30B500B9004830BE00AB
:100490007A30BF00C30803194E2A772A2030B300F0
:1004A000C4080319542A7A2A2030B400B500C508BC
:1004B00003195B2A7D2A2030B600C6080319612A79
:1004C000802A2030B700C7080319672A832A203002
:1004D000B800B900C80803196E2A862A2030BA006D
:1004E000C9080319742A892A2030BB008C2A4308C2
:1004F000303EB3004408303EB4004508303EB600FC
:100500004608303EB7004708303EB8004808303E45
:10051000BA004908303EBB004A08303EBC00072BF9
:100520004230B0003D30B1002030B200BD002E306E
:10053000B500B9004830BE007A30BF00CB080319BF
:10054000A22ACB2A2030B300CC080319A82ACE2A2D
:100550002030B400B500CD080319AF2AD12A2030CD
:10056000B600CE080319B52AD42A2030B700CF0828
:100570000319BB2AD72A2030B800B900D0080319C4
:10058000C22ADA2A2030BA00D1080319C82ADD2A83
:100590002030BB00E02A4B08303EB3004C08303E10
:1005A000B4004D08303EB6004E08303EB7004F084C
:1005B000303EB8005008303EBA005108303EBB0013
:1005C0005208303EBC00072B5330B0007730B100EA
:1005D0006530B2006530B3007030B4003D30B50016
:1005E0002030B600B700B800B900BA00BB00BC00AC
:1005F000F51F012B2030BD004F30BE004E30BF0034
:10060000072B4F30BD004630BE004630BF004223AE
:1006100008008312031385018601870183162730A2
:1006200081000130850003308600003087000C1007
:100630000C13FF309F0083121F1098139412101098
:100640001211F5100230C2000430D3000730D4007C
:10065000FF30F800F9000930FA00FF30C1004030E7
:10066000D5004B30D6004C30D7000030D800B83021
:10067000D9000B30DA000030DB000030DC00F5136D
:10068000751108008030AE00303084001030AF00AB
:100690002E087723AE0A00088123840AAF0B482B6B
:1006A000C030AE001030AF002E087723AE0A2030E5
:1006B0008123AF0B542B0800932393233030860003
:1006C0008D2393238D2393238D2393232030860022
:1006D0008D2393232830772393230C307723932380
:1006E0000130772393230630772393230800C0003B
:1006F000F03986008D23400EF03986008D23860167
:100700000800C000F039860006158D23400EF03930
:10071000860006158D23860108009B2386159B23E2
:1007200086119B2308001E30AF00AE01AE0B962B46
:10073000AF0B952B08001E30A000A00B9D2B0800CE
:100740002408A00725080318250FA1072608031869
:10075000260FA20727080318270FA307080024085D
:10076000A0022508031C250FA1022608031C260F42
:10077000A2022708031C270FA3020800230827064C
:100780000319C62BAD0023308400DD2B220826067A
:100790000319CE2BAD0022308400DD2B2108250665
:1007A0000319D62BAD0021308400DD2B2008240650
:1007B00003190034AD0020308400AD1FE22B801FF0
:1007C0002D342B342D1FE72B001F2D342B34AD1E61
:1007D000EC2B801E2D342B342D1EF12B001E2D34BE
:1007E0002B34AD1DF62B801D2D342B342D1DFB2BF2
:1007F000001D2D342B34AD1C002C801C2D342B34CB
:10080000001C2D342B3403102030A800A001A101BE
:10081000A201A301A401A501A601A701AA0DAB0D88
:10082000AC0DAD0DA00DA10DA20DA30DA80B312C8B
:10083000230E0F39A70023080F39A600220E0F3907
:10084000A50022080F39A400210E0F39A3002108AA
:100850000F39A200200E0F39A10020080F39A00087
:100860000800203084003E24213084003E242230C1
:1008700084003E24233084003E240E2C03300007E5
:10088000A900A919800030300007A900A91B800029
:100890000034E501E601E701E8016430A00007301B
:1008A000A100A201A301693084001E256508A400EF
:1008B0006608A5006708A6006808A700A02320080E
:1008C000E5002108E6002208E7002308E800883058
:1008D000A0000730A100A201A3016A3084001E25F8
:1008E0006508A4006608A5006708A6006808A700B8
:1008F000A0232008E5002108E6002208E7002308DD
:10090000E800AC30A0000730A100A201A3016B30C9
:1009100084001E256508A4006608A5006708A600D7
:100920006808A700A0232008E5002108E6002208A7
:10093000E7002308E800D030A0000730A100A201A2
:10094000A3016C3084001E256508A4006608A5007C
:100950006708A6006808A700A0232008E500210872
:10096000E6002208E7002308E800F430A000073082
:10097000A100A201A3016D3084001E256508A4001A
:100980006608A5006708A6006808A700A02320083D
:10099000E5002108E6002208E7002308E8001830F7
:1009A000A0000830A100A201A3016E3084001E2522
:1009B0006508A4006608A5006708A6006808A700E7
:1009C000A0232008E5002108E6002208E70023080C
:1009D000E8003C30A0000830A100A201A3016F3064
:1009E00084001E256508A4006608A5006708A60007
:1009F0006808A700A0232008E5002108E6002208D7
:100A0000E7002308E8006030A0000830A100A20140
:100A1000A301703084001E256508A4006608A500A7
:100A20006708A6006808A700A0232008E5002108A1
:100A3000E6002208E7002308E80008008008031DFC
:100A4000242DA001A1010800800D000DA400A40325
:100A5000A501A601A701A0232108031783128F0077
:100A60000313200803178D0083160C1400000000E8
:100A700083120C080313A8000130A400A501A601ED
:100A8000A701AF23200803178D00031321080317C4
:100A90008F0083160C140000000083120C0803134F
:100AA000A9000130A400A501A601A701AF232008D9
:100AB00003178D000313210803178F0083160C14EE
:100AC0000000000083120C080313AA000130A400E8
:100AD000A501A601A701AF23200803178D0003136A
:100AE000210803178F0083160C14000000008312E6
:100AF0000C080313AB000130A400A501A601A70157
:100B0000AF232808A0002908A1002A08A2002B086A
:100B1000A3000800061C932D411C992D861C962DC0
:100B2000C11C992D08004118992D8E2DC118992DA1
:100B30000800C10DC10D061C9F2D4114A02D4110B0
:100B4000861CA42DC114A52DC1104108E13A031D36
:100B5000AA2DAF2D4108D23A031D0800642E420889
:100B6000033A031DBB2DD30A5308053A031D55292B
:100B70000130D30055294208013A031DC72DD40A7C
:100B80005408093A031D94290130D40094294208DD
:100B9000023A031DFD2D5508A0005608A100570874
:100BA000A2005808A300EC26A023A4015930A500F8
:100BB0006230A6000230A700BE232B3A031DF02DA1
:100BC000A001D501AA015930A100D600AB006230C6
:100BD000A200D700AC000230A300D800AD00402F27
:100BE0002008D500AA002108D600AB002208D700B3
:100BF000AC002308D800AD00402F4208043A031D82
:100C00005D2E5908A0005A08A1005B08A2005C08EC
:100C1000A300EC26A0232008E5002108E600220816
:100C2000E7002308E800A0015A30A1006230A200CA
:100C30000230A3005508A4005608A5005708A600D6
:100C40005808A700AF232008A4002108A500220807
:100C5000A6002308A7006508A0006608A100670891
:100C6000A2006808A3002408E5002508E60026087D
:100C7000E7002708E800BE232B3A031D502E650825
:100C8000A000D900AA006608A100DA00AB0067083E
:100C9000A200DB00AC006808A300DC00AD00522F0E
:100CA0002008D900AA002108DA00AB002208DB00E6
:100CB000AC002308DC00AD00522F4208053A031DAA
:100CC0000800F51FF517E42A4208033A031D6D2EAC
:100CD000D30B55290430D30055294208013A031D8E
:100CE000762ED40B94290830D40094294208023A75
:100CF000031DAC2E5508A0005608A1005708A200FD
:100D00005808A300EC26BE232D3A0319912EAF23D9
:100D10001430A400A501A601A701BE232D3A031D8E
:100D20009F2E1430A000D500AA00A101D601AB016E
:100D3000A201D701AC01A301D801AD01402F2008C9
:100D4000D500AA002108D600AB002208D700AC00CD
:100D50002308D800AD00402F4208043A031DE22EBC
:100D60005908A0005A08A1005B08A2005C08A30073
:100D7000EC26BE232D3A0319C72EAF23FF30A40063
:100D8000A501A601A701BE232D3A031DD52EFF30D4
:100D9000A000D900AA00A101DA01AB01A201DB0188
:100DA000AC01A301DC01AD01522F2008D900AA003B
:100DB0002108DA00AB002208DB00AC002308DC00CD
:100DC000AD00522F4208053A031D0800F51FE42A22
:100DD000F513F5107515E42A01305406031DF62E9F
:100DE0000130A400A501A601A701080002305406A5
:100DF000031D002F0A30A400A501A601A7010800C9
:100E000003305406031D0A2F6430A400A501A60177
:100E1000A701080004305406031D152FE830A40074
:100E20000330A500A601A701080005305406031DE4
:100E3000202F1030A4002730A500A601A70108002C
:100E400006305406031D2C2FA030A4008630A500C8
:100E50000130A600A701080007305406031D382FF3
:100E60004030A4004230A5000F30A600A7010800C2
:100E70008030A4009630A5009830A600A701080095
:100E800003242708C3002608C4002508C500240839
:100E9000C6002308C7002208C8002108C90020088E
:100EA000CA003C2A03242708CB002608CC002508CA
:100EB000CD002408CE002308CF002208D00021084E
:100EC000D1002008D200902A00000000000022007B
:100ED0000000000000004400000000000000670067
:100EE0000000000000008900000000000000AB00CE
:100EF000000000000000CE00000000000000F00034
:100F00000000000001001200000000000100350098
:100F10000000000001005700000000000200AF00C8
:100F200000000000040006000000000005005E0054
:100F3000000000000600B5000000000008000D00E1
:100F40000000000009006500000000000A00BC006D
:100F5000000000000C001400000000000D006B00F9
:100F6000000000001A00D700000000002800430025
:100F7000000000003500AF000000000043001B002F
:100F80000000000050008700000000005D00F3003A
:100F9000000000006B005F00000000007800CB0044
:100FA0000000000086003700000001000C006F0008
:100FB000000001009200A700000002001800DE00FF
:100FC000000002009F0016000000030024005E00E5
:100FD00000000300AB008600000004003100BD00EB
:100FE00000000400B700F500000005003E002D00E1
:100FF00000000A007C005A0000000F00BA008800C0
:1010000000001400F800B50000001A003600E200ED
:1010100000001F007500100000002400B3003D0018
:1010200000002900F1006B0000002F002F00980045
:10103000000034006D00C50000006800DB008B007C
:1010400000009D00490051000000D100B7001700CA
:10105000010006002400DD0001003A009200A30018
:1010600001006F00000068000100A3006E002E0068
:101070000100D700DB00F40002000C004900BA00B8
:10108000040018009300740006002400DD002F0007
:10109000080031002600E9000A003D007000A300AE
:1010A0000C004900BA005E000E0056000400180053
:1010B000100062004D00D20012006E0097008D00FB
:1010C00014007A00E10047002800F500C2008F00FC
:1010D0003D007000A300D7005100EB0085001E000A
:1010E0005300770065006500700020004700650030
:1010F0006E0065007200610074006F0072002000D5
:101100005A0055004D0045005200200056003100A5
:101110002E00330061002000320030003100350025
:02400E00B23FBF
:00000001FF
